
 Start  Stop   Length Name                   Class
 00000H 0137FH 01380H CODER                  
 01380H 030CCH 01D4DH CODE                   
 030CDH 0344BH 0037FH DATA                   
 03450H 03517H 000C8H STACK                  

 Origin   Group
 0138:0   DG

  Address         Publics by Name

 0138:12D6       $M_CLS_1
 0138:13EA       $M_CLS_2
 0138:1484       $M_CLS_3
 0138:14B3       $M_CLS_4
 0138:1144       $M_MSGSERV_1
 0138:11C3       $M_MSGSERV_2
 0138:0930       amis_sign
 0000:04E8       BlkSiz
 0000:04AC       Buffer
 0000:04A6       BusyTick
 0000:0E97       close_dev
 0000:06A6       doint
 0000:0D4D       do_21
 0000:04EA       EndPtr
 0000:04A8       EndQueue
 0000:054F       EndRes
 0000:065D       enterprint
 0000:111D       FileQueue
 0138:07EA       GoDispMsg
 0000:0692       leaveprint
 0000:1166       ListName
 0000:04A5       MaxTick
 0000:0527       MESBAS
 0000:123C       MoveTrans
 0138:1F69       NameBuf
 0000:04C9       NxtChr
 0000:0E55       open_dev
 0000:04D0       PChar
 0000:04A7       QueueLen
 0000:1339       RealMove
 0000:0000       R_MES_BUFF
 0000:04A3       SliceCnt
 0138:0C10       SYSDISPMSG
 0138:0AC2       SYSGETMSG
 0138:094A       SYSLOADMSG
 0138:1568       SYSPARSE
 0000:04A4       TimeSlice
 0000:0DCA       TO_DOS
 0138:0534       TransRet
 0138:2198       TransSize

  Address         Publics by Value

 0000:0000       R_MES_BUFF
 0000:04A3       SliceCnt
 0000:04A4       TimeSlice
 0000:04A5       MaxTick
 0000:04A6       BusyTick
 0000:04A7       QueueLen
 0000:04A8       EndQueue
 0000:04AC       Buffer
 0000:04C9       NxtChr
 0000:04D0       PChar
 0000:04E8       BlkSiz
 0000:04EA       EndPtr
 0000:0527       MESBAS
 0000:054F       EndRes
 0000:065D       enterprint
 0000:0692       leaveprint
 0000:06A6       doint
 0000:0D4D       do_21
 0000:0DCA       TO_DOS
 0000:0E55       open_dev
 0000:0E97       close_dev
 0000:111D       FileQueue
 0000:1166       ListName
 0000:123C       MoveTrans
 0000:1339       RealMove
 0138:0534       TransRet
 0138:07EA       GoDispMsg
 0138:0930       amis_sign
 0138:094A       SYSLOADMSG
 0138:0AC2       SYSGETMSG
 0138:0C10       SYSDISPMSG
 0138:1144       $M_MSGSERV_1
 0138:11C3       $M_MSGSERV_2
 0138:12D6       $M_CLS_1
 0138:13EA       $M_CLS_2
 0138:1484       $M_CLS_3
 0138:14B3       $M_CLS_4
 0138:1568       SYSPARSE
 0138:1F69       NameBuf
 0138:2198       TransSize

Program entry point at 0138:0000
